:0200000480007A
:100000006F00C004732F2034930F8000630AFF0336
:10001000930F90006306FF03930FB0006302FF038A
:10002000170F0080130F0FFE63040F0067000F000F
:10003000732F203463540F006F004000136E9E53E3
:10004000171F00002320CFFD6FF09FFF732540F1A5
:100050006310050073251030635805000F00F00F82
:10006000130E100073000000130E00009702000032
:10007000938282F973905230735020307350303035
:1000800073504030970200809382C2F7638C020065
:10009000739052109302B01A739022307323203061
:1000A000E39E62F873500030970200009382420191
:1000B00073901234732540F1730020309306F006DC
:1000C00017250000031505F4972500008395A5F377
:1000D00013000000130000001300000013000000D4
:1000E00013000000130000001300000013000000C4
:1000F00013000000130000001300000013000000B4
:1001000097020000239AA200970200002397B200F2
:100110000F1000009386E60D13000000930EC01B25
:10012000130E2000639AD607130740061307F7FF44
:10013000E31E07FE970200002396A2049702000028
:100140002393B2040F1000001300000013000000FE
:100150001300000013000000130000001300000053
:100160001300000013000000130000001300000043
:100170001300000013000000130000001300000033
:100180009386B62213000000930E9030130E3000B9
:100190006394D601631CC0010F00F00F63000E00D2
:1001A000131E1E00136E1E00730000000F00F00FE0
:1001B000130E100073000000731000C00000000058
:1001C000000000000000000000000000000000002F
:1001D000000000000000000000000000000000001F
:1001E000000000000000000000000000000000000F
:0401F000000000000B
:1010000000000000000000000000000000000000E0
:1010100000000000000000000000000000000000D0
:1010200000000000000000000000000000000000C0
:1010300000000000000000000000000000000000B0
:081040000000000000000000A8
:102000009386D614000000000000000000000000CD
:040000058000200057
:00000001FF
